:1000000061288F00220884002009282084138F088B
:1000100003195C28F03091000E0880389000F03011
:1000200091030319910003198F0303195C28182801
:100030002B2003010C1820088E1F20088E0803199E
:100040000301900F252880060C28262800000F2881
:10005000841780055C280D080C0403198C0A803075
:100060000C1A8D060C198D068C188D060D0D8C0D35
:100070008D0D5C288F018E00FF308E07031C8F07CB
:10008000031C5C2803308D00DF3048203C288D01A4
:10009000E83E8C008D09FC30031C51288C070318A6
:1000A0004E288C0764008D0F4E280C1857288C1C86
:1000B0005B2800005B28080083130313831264008D
:1000C0000800831603308500013086008312061273
:1000D00083160612831206138316061383128612E2
:1000E00083168612831286108316861083120611D9
:1000F000831606118312861183168611053083122A
:10010000A2000830A00073308E000A300120323087
:100110008E000A3001200130A40064000630240261
:100120000318C428061683160612831206178316B0
:100130000613831201308F002C303B206400051819
:10014000A2289E280612831606128312061383160F
:1001500006138312861483168610831206158316DF
:100160000611831201308F002C303B20640085186B
:10017000BA28B628861083168610831206118316B5
:1001800006118312A40F8D280130A40064000630EC
:1001900024020318FD2806168316061283128616FB
:1001A00083168612831201308F002C303B206400AE
:1001B0000518DB28D728061283160612831286122A
:1001C00083168612831286148316861083120615F0
:1001D00083160611831201308F002C303B206400FF
:1001E0008518F328EF2886108316861083120611CF
:1001F000831606118312A40FC6280130A4006400E0
:1002000006302402031836290616831606128312B6
:10021000861683168612831201308F002C303B2005
:100220006400051814291029061283160612831279
:100230008612831686128312861483168610831202
:10024000861583168611831201308F002C303B20D7
:10025000640085182C29282986108316861083129D
:100260008611831686118312A40FFF280130A40083
:1002700064000630240203186F290616831606123E
:100280008312061783160613831201308F002C3059
:100290003B20640005184D294929061283160612D1
:1002A0008312061383160613831286148316861090
:1002B0008312861583168611831201308F002C302D
:1002C0003B206400851865296129861083168610F5
:1002D00083128611831686118312A40F38298B2866
:0402E000630070291E
:02400E00F53F7C
:00000001FF
